:020000040800F2
:10000000C008002029020008D52300088520000828
:100010002D2300081F040008E12A0008000000004A
:10002000000000000000000000000000FD240008A7
:100030002505000800000000852400081925000897
:10004000430200084302000843020008430200087C
:10005000430200084302000843020008430200086C
:10006000430200084302000843020008430200085C
:100070007504000843020008430200084302000818
:10008000430200084302000843020008430200083C
:10009000210400084302000843020008430200084C
:1000A000430200084302000843020008430200081C
:1000B000430200084302000843020008430200080C
:1000C00043020008430200084302000843020008FC
:1000D000430200084302000843020008A92A00085E
:1000E00043020008430200084302000843020008DC
:1000F00043020008430200084302000843020008CC
:1001000043020008430200084302000843020008BB
:1001100043020008430200084302000843020008AB
:10012000430200084302000843020008430200089B
:10013000430200084302000843020008430200088B
:10014000430200084302000843020008430200087B
:10015000430200084302000843020008430200086B
:10016000430200084302000843020008430200085B
:100170004302000843020008430200080000000098
:10018000430200084302000800F002F800F03CF8C7
:100190000AA090E8000C82448344AAF10107DA45E2
:1001A00001D100F031F8AFF2090EBAE80F0013F0F8
:1001B000010F18BFFB1A43F001031847942B0000EE
:1001C000B42B0000103A24BF78C878C1FAD852077F
:1001D00024BF30C830C144BF04680C6070470000C1
:1001E0000023002400250026103A28BF78C1FBD840
:1001F000520728BF30C148BF0B6070471FB502F0DF
:1002000091FD1FBD10B510BD00F0CFF81146FFF7EE
:10021000F5FF02F0C7FC00F0EDF803B4FFF7F2FFC2
:1002200003BC00F0F5F80000094880470948004782
:10023000FEE7FEE7FEE7FEE7FEE7FEE7FEE7FEE796
:10024000FEE7FEE704480549054A064B70470000F3
:10025000B125000889010008C0020020C008002064
:10026000C0040020C004002053EA020C00F06980A2
:100270002DE9F04B4FF00006002B1FBFB3FA83F5BA
:1002800003FA05F424FA05F65E4012BF1643B2FAEB
:1002900082F502FA05F4C5F120051EBF22FA05FC1D
:1002A00044EA0C04203556EA044C4FEA144418BFC3
:1002B000641C4FF000084FF00009904271EB030CF2
:1002C00039D3002919BFB1FA81F701FA07F6B0FA5C
:1002D00080F700FA07F6C7F120071EBF20FA07FCD7
:1002E00046EA0C062037B6FBF4FCA7EB0507103FE7
:1002F00007F01F0BCBF120060CFA0BFB2CFA06F6CD
:1003000044BFB3460026202FA4BF5E464FF0000B2B
:100310005BEA060C08BF4FF0010B19EB0B09ABFBB6
:10032000027C48EB0608C01B06FB02CC0BFB03CC8F
:1003300071EB0C01C1E70B46024641464846BDE859
:10034000F08B13B54FF000004FF00001AFF30080C9
:10035000BDE81C4070474FF0000200B513469446BC
:100360009646203922BFA0E80C50A0E80C50B1F10D
:100370002001BFF4F7AF090728BFA0E80C5048BF21
:100380000CC05DF804EB890028BF40F8042B08BFBF
:10039000704748BF20F8022B11F0804F18BF00F8BB
:1003A000012B7047704770477047754600F02CF876
:1003B000AE4605006946534620F00700854618B052
:1003C00020B5FFF73FFFBDE820404FF000064FF09B
:1003D00000074FF000084FF0000B21F00701AC467A
:1003E000ACE8C009ACE8C009ACE8C009ACE8C00999
:1003F0008D46704710B50446AFF300802046BDE837
:100400001040FFF70ABF0000004870475C02002060
:1004100001491820ABBEFEE7260002007047FEE748
:10042000014800F02CBA00004401002038B50E4C01
:1004300040F2FF1525600025A560E56008252561CF
:100440000A4C050A25706070080AA070E170100A55
:1004500020716271180AA071E3716B46224602494D
:10046000034800F0ADF838BD2C0100200A00002040
:1004700044010020014800F091BC0000FC01002074
:1004800001681823CAB2103AB2FBF3F2054B6FF3BE
:100490000901032A9B5CC36500D9091D81650846D3
:1004A000704700002E2D000810B5014600208B6912
:1004B0008A6A4FF0C07453B1B3F5005F15D072B1C2
:1004C000012A0CD0022A0AD0032A09D104E01AB169
:1004D000012A06D0022A03D1C96AC90100D5012028
:1004E00010BDC96AA142FAD010BD002AF7D0012A76
:1004F000F2D0022AF3D0032AF3D010BD30B504683D
:10050000256825F480252560046863608368402B96
:10051000036803D099600068C26030BD9A600068CB
:10052000C16030BD7047000070EE202ADFED181A60
:100530009FED182A30EE600AF0EE623A41EE612A31
:1005400041EE213A00B5002083EE823AF0EE403AC7
:1005500001EE210A41EE613AC3EE820AC2EE823A0E
:1005600080EE021AB0EE430A01F0CAFFB0EE600A54
:10057000012001F0C5FFB0EE630A022001F0C0FFC8
:10058000B0EE410A03205DF804EB01F0B9BF0000B2
:100590001F85AB3E3333333E72B6FEE790F8202022
:1005A000012A07D0022A05D0416A41F48021416224
:1005B00001207047006842690A4342610020704789
:1005C000F0B590F820500468A468012D05D0022DE4
:1005D00003D0416A41F480214DE014F0406F01D115
:1005E000E50045D5C4F301640125A5401D608D6873
:1005F0004FF4C0739DB1CE6835434E6845EAC605D9
:10060000066803EB0417F5514FF4C275076805EB54
:1006100004150E697E51097D012905D009E00E8877
:10062000CD6845EA4655EBE701684E5946F48076B9
:100630004E511179D2F805504FF4C67641EA0521A2
:10064000056806EB0416A9511178D2F801204FF481
:10065000C47541EA0221026805EB04155151006896
:1006600003EB0411425842F0010242500020F0BD59
:10067000416A41F4001141620120F0BD10B590F8CB
:100680002020012A07D0022A05D0416A41F48021A6
:100690004162012010BD3B48D0F8002242F0010227
:1006A000C0F80022D0F8002222F47C52C0F80022C8
:1006B000D0F800224B6A42EA0322C0F800220A7DE9
:1006C00002F01F0301229A40D0F81C329343C0F875
:1006D0001C32CB69B3B9D0F80C329343C0F80C325A
:1006E0008C894B6864F31F434C6900EBC404C4F865
:1006F00040320C890B6864F31F434C6900EBC4045F
:10070000C4F84432CB69012B16D1D0F80C32134314
:10071000C0F80C320C884B6864F31F434C6900EB43
:10072000C404C4F840320C89CB6864F31F434C699D
:1007300000EBC404C4F844328B69002BD0F80432B7
:100740000ED01343C0F804320B69002BD0F81432DA
:1007500008D01343C0F81432096A012904D008E014
:100760009343EFE79343F5E7D0F81C121143C0F829
:100770001C12D0F8001221F00101C0F80012002074
:1007800010BD000000640040704770B590F8204034
:10079000012C05D0022C03D0416A41F4802128E0CD
:1007A000046809B32469A40720D04FF4D8740568FD
:1007B00004EB01142D5915F00405956005682D59B9
:1007C0001AD0ED08556005682C5904F00204D46075
:1007D0004FF4DA74056804EB01142E5906F00F0685
:1007E000082E0CD308250DE0E468DCE7416A41F4EB
:1007F00000114162012070BD6D0D1560E3E72D59B8
:1008000005F00F05156105682D59C5F3072595619C
:1008100005682C59240C54614FF4DC72046802EB17
:100820000112A4581C700468A458240A5C7004685F
:10083000A458240C9C700468A258120EDA704FF46D
:10084000DE72046802EB0112A4581C710468A458FB
:10085000240A5C710468A458240C9C710468A25892
:10086000120EDA71006829B1016941F020010161BD
:10087000002070BDC16841F02001C160F8E72DE99A
:10088000F05F0546006800244669D0F80490876848
:10089000D0F80CB0D0F810A0D0F81880F10748D0EC
:1008A000F90714D001218160B80703D5284600F06C
:1008B00014FA0CE0780702D54FF4006407E038071B
:1008C00002D54FF4805402E0284600F005FAF805FE
:1008D00016D529684FF480708860B80503D528467E
:1008E00000F0FDF90CE0780502D544F4005407E06F
:1008F000380502D544F4804402E0284600F0EEF9C1
:10090000F80316D529684FF480308860B80303D502
:10091000284600F0E6F90CE0780302D544F40044E0
:1009200007E0380302D544F4803402E0284600F0A2
:10093000D7F9300707D55FEACB6004D529681020C6
:1009400044F40074C86070074FF0080707D55FEAE9
:100950000B7004D52868C760284600F057F9B00727
:1009600006D52868C068800702D0284600F050F9F4
:10097000700607D55FEACA6004D52968102044F4E0
:1009800080640861B00607D55FEA0A7004D528685C
:100990000761284600F070F9F00606D5286800695E
:1009A000800702D0284600F068F9B00308D55FEA56
:1009B000C96005D5296810204860284600F05EF916
:1009C000F00307D55FEA097004D528684760284618
:1009D00000F088F9300446D55FEA497040D5F0054B
:1009E00004D55FEAC87001D044F00104B00504D515
:1009F0005FEA887001D544F00204700504D55FEA0F
:100A0000487001D544F00404300529D518F0700F62
:100A100026D008F07000402815D006DC102809D038
:100A200020280AD0302816D10AE050280ED060289D
:100A300011D10EE044F008040DE044F010040AE087
:100A400044F0200407E044F0400404E044F0800453
:100A500001E044F480742868816921F070018161AB
:100A6000296804204860002C05D0686A2043686229
:100A70002846FFF789FEBDE8F09F70B5040003D05B
:100A800094F8200010B104E0012070BD204600F071
:100A900081F82068016841F00101016000F0ECFB81
:100AA0000546052604E000F0E7FB401B0A2811D8A4
:100AB00020684068C007F6D02068016821F0020174
:100AC000016000F0D9FB05460BE000F0D5FB401BB0
:100AD0000A2806D9606A40F40030606284F8206019
:100AE000D2E7206840688007EFD4207E0128206884
:100AF00001683DD021F080010160607E01282068FE
:100B0000016838D021F040010160A07E01282068F2
:100B1000016833D021F020010160E07E01282068C7
:100B200001682ED041F010010160207F012820686B
:100B3000016829D021F008010160607F0128206848
:100B4000016824D021F004010160D4E902010843C6
:100B5000D4E90412114308436168491E084321681F
:100B6000C86100206062012084F82000002070BD70
:100B700041F08001C0E741F04001C5E741F02001AC
:100B8000CAE721F01001CFE741F00801D4E741F0B6
:100B90000401D9E710B586B0044614216846FFF772
:100BA000DAFB17492068884227D1164800210268DD
:100BB00042F000720260006800F000700590114879
:100BC0001038026842F0080202600068022200F059
:100BD000080005900320CDE90210CDE900020920AC
:100BE00004906946084800F049FA00221146142092
:100BF00000F0B0FB142000F09FFB06B010BD000019
:100C00000064004040380240000C02407047000081
:100C100010B58CB002AB04AA0021FFF7B6FD049812
:100C2000012805D0022803D0032801D004281DD1B3
:100C3000401E0F49C0B20F4A087000EB800302EB60
:100C4000430132F813400C81BDF8084064BA22F821
:100C50001340BDF80A2052BA4A80BDF80C2052BA9F
:100C60008A809DF80E208A7101F02AFF0CB010BD19
:100C700000000020300000207047704770470000DF
:100C800070B5044690F82000012804D0606A40F452
:100C90000020606218E0022084F8200020680168CB
:100CA00021F00101016000F0E7FA05460EE000BF07
:100CB00000F0E2FA401B0A2808D9606A40F40030CC
:100CC0006062052084F82000012070BD2068406823
:100CD000C007EDD1606270BD7047704770477047C4
:100CE0007047704770472DE9F0410446876D00F06A
:100CF000C3FA064694F835000025022806D0802065
:100D0000606584F834500120BDE8F08120680168F6
:100D100021F0160101602068416921F080014161E4
:100D2000206C08B9A06C20B12068016821F008018E
:100D300001602068016821F0010101600CE000F011
:100D40009BFA801B052807D920206065032084F8C2
:100D5000350084F83450D7E720680068C007EED12A
:100D600094F85C103F208840B860012084F835007A
:100D700084F834500020C7E790F83510022903D0DA
:100D80008021416501207047052180F835100068F9
:100D9000016821F001010160002070472DE9F8434E
:100DA00004464FF00009CDF8009063484FF4165107
:100DB000A56D0068B0FBF1F72E6894F85C10082070
:100DC00000FA01F131420FD021680A6852070BD5B1
:100DD0000A6822F004020A6094F85C108840A86057
:100DE000606D40F00100606594F85C104FF0010800
:100DF00008FA01F0304208D021684969090604D593
:100E0000A860606D40F00200606594F85C100420FA
:100E10008840304208D021680968890704D5A86055
:100E2000606D40F00400606594F85C10102088400C
:100E3000304218D021680968090714D5A8602068D5
:100E40000168490304D50068000308D5A16C07E0D8
:100E50000168C90503D4016821F008010160216C13
:100E600009B12046884794F85C1020208840304221
:100E700031D021680968C9062DD5A86094F83500DD
:100E800005282068016806D0490347D5006800039B
:100E90001DD4616C1CE021F01601016020684169DD
:100EA00021F080014161206C08B9A06C20B120685C
:100EB000016821F00801016094F85C103F2088402F
:100EC000A86084F8358084F83490216D1FE0E16BD0
:100ED00009B120468847606D00282BD0606DC0079F
:100EE00014D0052084F835002068016821F0010144
:100EF00001600098401C0090B84203D82068006848
:100F0000C007F6D184F8358084F83490E16C00296C
:100F100010D001B02046BDE8F04308470168C9057C
:100F2000D5D4016821F01001016084F8358084F87F
:100F30003490CCE7BDE8F883200000202DE9F04193
:100F4000044600F099F906465CB1022084F83500A9
:100F5000002584F834502068016821F00101016007
:100F60000DE00120BDE8F08100F086F9801B052826
:100F700005D920206065032084F83500F2E7206859
:100F80000068C007F0D12268116820480140D4E908
:100F900001031843D4E90336334318436369184304
:100FA000A3691843E3691843236A18430843616A35
:100FB000042903D1D4E90B131943084310602068B6
:100FC0004069666A20F0070130460E430127042875
:100FD0000CD1A06A0643E06A40B12046FFF764FAEC
:100FE00020B14020606584F83570BAE7206846611A
:100FF0002046FFF745FA94F85C203F21914081603C
:10100000656584F835700020ACE700003F8010F083
:1010100070B5044690F83400002501280CD001205A
:1010200084F8340094F835600020012E06D084F84E
:1010300034000225284670BD022070BD022684F8C7
:10104000356060652046FFF759FA2068016841F075
:1010500001010160EEE7000070B5044600F00CF9F4
:101060000546601C02D004480078044400F004F9EE
:10107000401BA042FAD370BD140000202DE9F84FA8
:10108000DFF8BCA10022012503264FF00F090AF169
:10109000040BAAF1040E00BF0B6805FA02F423400A
:1010A000A34270D10F7907F00307012F01D0022F5F
:1010B00016D187684FEA420806FA08FC27EA0C07AF
:1010C000D1F80CC00CFA08FC4CEA070CC0F808C0B8
:1010D0004768A7430C79C4F3001494403C43446030
:1010E0000C79E443A4070AD0C4684FEA420C06FA1C
:1010F0000CF7BC438F6807FA0CF72743C7600C79DD
:1011000004F00304022C12D1D40800EB840CDCF8A8
:1011100020405707FF0E09FA07F824EA0804D1F81F
:10112000108008FA07F848EA0408CCF82080046820
:101130004FEA420C06FA0CF7BC430F7907F003079D
:1011400007FA0CF7274307604C6814F4403F70D04F
:101150003C4C276847F480472760246822F0030747
:1011600004F480440094384C07EB040CDCF8084885
:1011700097074FEA177809FA08F7BC43334FB8428C
:1011800002D1002724E054E0314FB84201D10127B9
:101190001EE0304FB84201D1022719E02E4FB8426D
:1011A00001D1032714E02D4FB84201D104270FE0ED
:1011B0002B4FB84201D105270AE02A4FB84201D18E
:1011C000062705E0284FB84201D1072700E008278D
:1011D00007FA08F72743CCF80878DAF800405746B2
:1011E000D1F804C09C435FEACC2C00D51C433C6082
:1011F000DBF800405F46D1F804C09C435FEA8C2CCA
:1012000000D51C433C60DEF800407746D1F804C0AE
:101210009C435FEA8C3C00D51C433C60084F083F70
:101220003C68D1F804C09C435FEACC3C00D51C4329
:101230003C60521C102AFFF42FAFBDE8F88F00006D
:10124000083C0140443802400030014000000240A8
:101250000004024000080240000C0240001002405E
:101260000014024000180240001C02400AB18161D3
:1012700070470904FBE700000148806870470000E0
:101280001400002002488168027811448160704790
:10129000140000200B4810B5016841F40071016092
:1012A000016841F480610160016841F4807101606E
:1012B000032000F06FF80F2000F006F800F024F88B
:1012C000002010BD003C024070B50D4D04464FF4A7
:1012D0007A712878B1FBF0F00A490968B1FBF0F0A7
:1012E00000F00CFB48B9102C07D200222146501EFA
:1012F00000F030F800206C6070BD012070BD00006F
:1013000014000020200000200A4808B5016841F4BC
:1013100080410160006800F4804000900548001F93
:10132000016841F080510160006800F08050009039
:1013300008BD000044380240002809DB00F01F020D
:10134000012191404009800000F1E020C0F8001127
:1013500070470000F0B40E4B1B680C46C3F3022329
:10136000C3F10705042D00D90425191D072901D251
:10137000002300E0DB1E012606FA05F1491E21408C
:1013800099409E40761E16403143F0BC01F0A9BB47
:101390000CED00E0064900F0070208684FF6FF0375
:1013A000184040EA0220034A1043086070470000DA
:1013B0000CED00E00000FA052DE9F0470E460500AF
:1013C00065D0DFF81481D8F80000F7B200F007000C
:1013D000B04207D288F80070D8F8000000F007008B
:1013E000B04254D128683D4C810712D5400703D53F
:1013F000206840F4E05020602878000703D520687A
:1014000040F4604020602068A96820F0F0000843A4
:1014100020602878C0072DD0304968680839012835
:1014200012D0022813D0032811D009688907002997
:101430002DDA216821F0030101432160FFF71CFF31
:10144000814641F2883A0EE009688903EFE70968AE
:101450008901ECE7FFF710FFA0EB0901514502D924
:101460000320BDE8F0872068696800F00C00B0EB4D
:10147000810FEFD1D8F80010404601F00701B142CA
:1014800007D90770006800F00700B04201D00120C2
:10149000E7E72878400705D52068E96820F4E050A0
:1014A000084320602878000706D52068296920F4C1
:1014B000604040EAC100206000F038F82168084A26
:1014C000C1F30311515CC840064908600648006832
:1014D000FFF7FAFE0020C4E7003C02400838024053
:1014E000362D00082000002018000020044805497F
:1014F00000680968044AC1F38221515CC840704702
:101500002000002008380240462D00080448054904
:1015100000680968044AC1F34231515CC840704711
:101520002000002008380240462D0008154810B55C
:10153000006810F00C02144813D01449042A0FD08C
:10154000082A0ED10F4C241F2268236802F03F02A4
:101550005B0207D52068C0F38810A0FB010106E0FC
:10156000084610BD2168C1F38811A1FB00010023CA
:10157000FEF77AFE2168C1F30141491C4900B0FB26
:10158000F1F010BD083802400024F40040787D01DD
:101590002DE9F84F04006ED02078DFF84C93C00797
:1015A000A9F104054AD009F104000168C1F38101E1
:1015B000012908D00068C0F3810002280AD1D9F8B7
:1015C0000000400206D52868800337D560680028EF
:1015D000E1D033E06068B0F5803F10D0B0F5A02FC7
:1015E000286810D020F480302860286820F48020FB
:1015F00028606068A8B1FFF73FFE06460DE0286846
:1016000040F48030F4E740F480202860F7E700BF22
:10161000FFF732FE801B642873D828688003F7D553
:101620000CE0FFF729FE064605E000BFFFF724FEA9
:10163000801B6428F0D828688003F7D42078DFF86E
:10164000AC8280074FF0000A3ED5A748001D016814
:1016500011F00C0F08D00068C0F3810002280BD1F4
:10166000D9F80000400207D42868800716D5E06842
:10167000012800D112E033E1E068B8B10120C8F8D8
:101680000000FFF7F9FD064605E000BFFFF7F4FD97
:10169000801B0228C0D828688007F7D528682169F0
:1016A00020F0F80040EAC10028600DE0C8F800A072
:1016B000FFF7E2FD064604E0FFF7DEFD801B02288F
:1016C0001FD828688007F7D42078000722D5864FD6
:1016D00087486169703771B101210160FFF7CCFD66
:1016E000064604E0FFF7C8FD801B022809D83868C9
:1016F0008007F7D50EE0C0F800A0FFF7BDFD064655
:1017000005E082E0FFF7B8FD801B02287DD838682D
:101710008007F7D42078400768D5DFF8CCB10027E0
:101720000BF13C0BDBF80000C0000BD4DBF8001021
:1017300041F08051CBF80010DBF80000012700F0E9
:10174000805000906B4E3068C00510D4306840F473
:1017500080703060FFF790FD009005E0FFF78CFD92
:101760000099401A022850D83068C005F6D55E4E60
:10177000A0686C3601280FD00528306810D020F002
:1017800001003060306820F004003060A068B8B11B
:10179000FFF772FD00900FE0306840F00100F4E7C1
:1017A00040F004003060F7E7FFF766FD0099411A4A
:1017B00041F28830814266D830688007F4D50EE067
:1017C000FFF75AFD009007E0FFF756FD0099411A18
:1017D00041F28830814256D830688007F4D42FB166
:1017E000DBF8001021F08051CBF80010A069C8B3DD
:1017F0003D49091D0968C1F3810102294AD0022827
:10180000504607D0C8F8600000E03CE0FFF734FD28
:1018100004463BE04746C8F86000FFF72DFD06464A
:1018200005E000BFFFF728FD801B02282BD82868A1
:101830008001F7D4D4E907010843A16A2E4A490878
:1018400002EB0141626A41EA8211084394F82C10CC
:1018500040EA0161C9F8001001203866FFF70CFD6D
:10186000044606E03EE000BFFFF706FD001B02282D
:1018700009D828688001F7D534E000BFFFF7FCFCE9
:10188000001B022802D90320BDE8F88F28688001D8
:10189000F4D427E00128F7D0D9F80000E26900F479
:1018A000800191421CD1226A00F03F01914217D180
:1018B00047F6C071626A0140B1EB821F10D1A26A83
:1018C0004FF0FF3300F4403103EB5202B1EB024F13
:1018D00006D194F82C1000F07060B0EB016F01D0CD
:1018E0000120D1E70020CFE7043802400000474242
:1018F000800E4742007000400000FFFF10B5401E00
:10190000B0F1807F01D3012010BD4FF0E024606171
:101910000F21601701F0E5F80020A0610720206189
:10192000002010BD10B590F83C20012A22D00122E1
:1019300080F83C20CA688C6822F4407222434C68CC
:1019400022F4806222430C6822F4006222430C6974
:1019500022F4805222434C6922F400522243C96986
:10196000002322F480420A4301684A6480F83C3034
:10197000002010BD022010BD70B590F83C20012A57
:1019800032D0012480F83C40022280F83D200368D8
:101990005A689D6822F070060A6832435A60134BF9
:1019A00002689A4214D0B2F1804F11D0104B9A4283
:1019B0000ED0104B9A420BD00F4B9A4208D00F4BCF
:1019C0009A4205D00E4B9A4202D00E4B9A4204D155
:1019D000496825F080031943916080F83D4000215B
:1019E00080F83C10084670BD022070BD0000014028
:1019F0000004004000080040000C004000040140CA
:101A0000004001400018004010B5040003D094F8D5
:101A10003D0010B107E0012010BD002084F83C001B
:101A2000204600F01FF8022084F83D00211D2068A8
:101A300000F0C6FD012084F8460084F83E0084F8DA
:101A40003F0084F8400084F8410084F8420084F8A4
:101A5000430084F8440084F8450084F83D000020E9
:101A600010BD000008B500680649884208D1064844
:101A7000016841F001010160006800F00100009080
:101A800008BD0000000001404438024070B5044623
:101A900090F83C000025012817D0012684F83C600E
:101AA000022084F83D002068826822F0770222F448
:101AB0007F4282600868502838D00DDC20284FD043
:101AC00005DC90B3102811D14AE0022070BD302807
:101AD00046D040280AD13BE060282FD070280DD096
:101AE000B0F5805F03D0B0F5005F12D0012584F817
:101AF0003D60002084F83C00284670BDCB68D1E9E9
:101B00000121206800F0C4FD2068816841F0770160
:101B100009E0CB68D1E90121206800F0B9FD206817
:101B2000816841F480418160E1E719E0CA68496851
:101B3000206800F081FE5021206806E0CA684968EC
:101B4000206800F08AFE6021206800F0ABFDCEE73F
:101B5000CA684968206800F06FFE40212068F4E7F9
:101B6000226801461046F0E710B586B004461421FD
:101B70006846FEF7F0FB0E492068884216D10D48F2
:101B80000021026842F010020260006800F01000BC
:101B900005904FF4007000900220CDE90101012072
:101BA000CDE9031069460448FFF768FA06B010BD96
:101BB00000000140303802400010024070B5044679
:101BC00090F83C0000260D4601280FD0012084F833
:101BD0003C006AB1042A1DD0082A2FD00C2A3FD01D
:101BE0000126002084F83C00304670BD022070BD04
:101BF000206800F05FFD2068816941F00801816183
:101C00002068816921F004018161206881692A6965
:101C1000114311E0206800F07DFD2068816941F4E6
:101C2000006181612068816921F48061816120689F
:101C300081692A6941EA02218161D2E7206800F0C6
:101C40009FFD2068C16941F00801C1612068C16938
:101C500021F00401C1612068C1692A69114311E0C2
:101C6000206800F0C1FD2068C16941F40061C161D4
:101C70002068C16921F48061C1612068C1692A6955
:101C800041EA0221C161ACE710B5040003D094F829
:101C90003D0010B107E0012010BD002084F83C0099
:101CA000204600F01EF8022084F83D00211D206827
:101CB00000F086FC012084F8460084F83E0084F899
:101CC0003F0084F8400084F8410084F8420084F822
:101CD000430084F8440084F8450084F83D00002067
:101CE00010BD704770477047F8B501680446086832
:101CF000CA684B6910F00F0F4FF0000559D003F080
:101D0000010602F49077374365D0C10705D0D105AD
:101D100003D5616C41F001016164410705D5D90724
:101D200003D0616C41F002016164810705D5D907D8
:101D300003D0616C41F004016164010707D502F032
:101D40002001314303D0616C41F008016164616C92
:101D500000293AD0800604D5900602D5204600F02E
:101D6000BCFD20684069616CC0F38010090700D495
:101D700060B3204600F08AFD20684069400621D506
:101D80002068143050E8001F21F0400140E80012A4
:101D9000002AF5D1E06BA8B172490165E06BFEF74E
:101DA000EBFF002811D0E06B016D01B0BDE8F04001
:101DB000084783060FD593060DD52046BDE8F840A9
:101DC00000F08BBD2046FFF78EFFF8BD2046FFF7E1
:101DD0008AFF6564F8BD266B2023012E7ED1C606DE
:101DE0007CD5D6067AD508684868009048694FF0D7
:101DF000020640064DD5E26B106840684FF48077CC
:101E00000004000C3AD0A18D814237D9E085D06919
:101E1000B8422DD020680C3050E8001F21F48071AA
:101E200040E80012002AF5D12068143050E8001F65
:101E300021F0010140E80012002AF5D12068143099
:101E400050E8001F21F0400140E80012002AF5D1BF
:101E500084F84230256320680C3050E8001F21F0E0
:101E6000100140E80012002AF5D1E06BFEF73BFFBD
:101E70006663A08DE18D401A81B206E0A18D81429A
:101E8000A8D1D069B842A5D166632046FFF72AFFE2
:101E9000F8BDA08DE18D401A81B2E08D0028F7D009
:101EA0000029F5D020680C3050E8002F22F4907201
:101EB00040E80027002FF5D12068143050E8002FAB
:101EC00022F0010240E80027002FF5D184F84230CB
:101ED000256320680C3050E8002F00E006E022F077
:101EE000100240E80023002BF3D1CDE705062BD5E7
:101EF000150629D594F841002128C9D1A068B0F56C
:101F0000805F01D12069B0B1206A411C2162216843
:101F100000784860E08C401E0004000CE084B7D1DB
:101F20002068C16821F08001C1602068C16841F06B
:101F30004001C160F8BD206A0088C0F30800486015
:101F4000206A801C2062E5E74006F3D55006F1D5F3
:101F5000CA68204622F04002CA6084F8413000F08E
:101F600090F8F8BD7F28000870B5040004D094F8FC
:101F70004100002510B106E0012070BD84F84050FA
:101F8000204600F023F8242084F841002068C1682E
:101F900021F40051C160204600F000FD2068016975
:101FA00021F4904101612068416921F02A014161D9
:101FB0002068C16841F40051C1606564202084F844
:101FC000410084F842006563002070BD70B586B0A2
:101FD000064614216846FEF7BEF924493068884257
:101FE00041D123480025016841F480210160006847
:101FF00000F4802005901E481038016841F004016B
:1020000001600068694600F0040005904FF44060EC
:1020100000900220CDE901050320039007200490E1
:102020001448FFF72BF8154C134820604FF0006060
:10203000C4E901054014C4E9035080106561C4E996
:102040000650256220466562FEF778FF08B1FEF76C
:10205000A3FAF463002211462720A663FFF77AF95A
:102060002720FFF769F906B070BD00000048004066
:10207000403802400008024028600240FC01002075
:1020800070477047FEE700000F4810B50D4901602A
:102090000321416000214FF410228160C0E9031246
:1020A0004FF400124261017641768176C176017764
:1020B0004177FEF7E2FC002803D0BDE81040FEF7B0
:1020C0006BBA10BD0064004044010020094808B507
:1020D000016841F4001101600068002200F4001062
:1020E000009011460C20FFF735F9BDE808400C20A0
:1020F000FFF722B9303802402DE9F04786B01421AD
:102100006846FEF728F934480024016841F00101CF
:102110000160016801F001010591016841F00801C9
:102120000160016801F008010591016841F00401B6
:102130000160016801F004010591016841F080012E
:102140000160016801F080010591016841F0100112
:1021500001600068DFF8848000F010004FF4007523
:102160000590002229464046FFF780F8DFF870907E
:102170004FF4C056002231464846FFF777F8DFF8A3
:1021800064A0AF00002239465046FFF76FF8009573
:102190000125CDE90154694640460394FEF76EFFE0
:1021A0000096CDE90154694648460394FEF766FF60
:1021B000A802CDE90004694648460294FEF75EFF96
:1021C0000097CDE90154694650460394FEF756FF47
:1021D00006B0BDE8F0870000303802400000024041
:1021E000001C02400010024010B596B000240F946D
:1021F00010941194129413941C2108A81494FEF7BF
:10220000AAF820216846FEF7A6F82848264901606A
:102210004721C0E901146321C0E9031444618461CA
:10222000FFF7F2FB08B1FEF7B7F94FF480500F90BB
:102230000FA91E48FFF72AFC08B1FEF7ADF91B48AD
:10224000FFF722FD08B1FEF7A7F9139413A9174869
:102250001494FFF791FB08B1FEF79EF96020CDE9D9
:1022600008040A940B940C940D94002208A90F48BA
:102270000E94FFF7A3FC08B1FEF78EF900944FF41B
:102280000050CDE904400294019403946946074844
:102290000794FFF747FB08B1FEF77EF90348FFF705
:1022A00063FC16B010BD0000000001406C0100206E
:1022B0000C4810B50A4901600B494160002181605A
:1022C0000C22C160C0E904128161C161FFF74CFEBC
:1022D000002803D0BDE81040FEF75EB910BD000035
:1022E00000480040B4010020A08601004FF4257191
:1022F000884202DC4942884201DA084606E000F1E1
:102300003101622902D89FED070A704700EE900A5A
:10231000DFED051AB8EEE01AC1EE210A20EE800AC0
:10232000704700000000000000002544FEE70000A8
:1023300000B5DFED112A114A9FED114ADFED114A78
:10234000F1EE043AB6EE003A002100BF01EB410085
:1023500002EB0010B0EE442AF0EE641AB0EE621AFE
:10236000F0EE430AB0EE630A0C3000F079F8491C35
:102370000429EBDB00BD0000CDCCCC3D5800002093
:1023800000007A4600007A4410B5104B104CB0EEB5
:10239000403A002101EB410003EB0012B2F90200C8
:1023A00000F096F892ED0B1A02F10C00F0EE430AE1
:1023B00031EE400A00F00FF8BDEEC00A10EE100A30
:1023C00024F81100491C0429E4DB10BD580000204A
:1023D00002000020FEE790ED001A21EE002A90EDA9
:1023E000031A00EE201A80ED031AD0ED061AB4EE9F
:1023F000E11AF1EE10FA06DCF1EE611AB4EEE11A20
:10240000F1EE10FA01D2C0ED031A90ED011AD0EDF1
:10241000031AD0ED042A21EE211A70EE622AD0EDC3
:10242000021A80ED040A32EE010A61EEA22AC2EE1F
:10243000A01A30EE210A80ED050AD0ED070AB4EEAD
:10244000E00AF1EE10FA06DCF1EE600AB4EEE00A02
:10245000F1EE10FA01D2C0ED050A90ED050A7047C1
:1024600080EC030A9FED060A80ED030A80ED040A62
:1024700080ED050AC0ED061A80ED072A70470000BE
:102480000000000070470000104A00B5B2F90400D7
:10249000B0EE000AFFF72AFFF0EE402AB2F906007C
:1024A000B0EE000AFFF722FFB0EE402AB2F90000BA
:1024B000B0EE080AFFF71AFFB0EE401AF0EE420A3B
:1024C000B0EE620A5DF804EBFEF72EB8240000209F
:1024D00000EE100AF0EE000A9FED071AB8EEC00AEF
:1024E00020EE200ADFED030A60EE200A80EE810A6A
:1024F00070470000DB0F4940000070427047000049
:10250000042806D2034900EB400001EB001080EDE7
:102510000B0A704758000020FEF7B4BE30B593B0E8
:1025200030216846FDF717FF14210CA8FDF713FFB3
:102530001D480025016841F080510160006800F0ED
:10254000805011901948016841F480410160006891
:10255000022400F480401190012003901020049088
:10256000009406940820CDE90750A820CDE909047D
:1025700004200B906846FFF70BF808B172B6FEE72F
:102580000CA90F2081E831004FF4A0500F904FF4B8
:102590008050109005210CA8FEF70EFF002801D0F6
:1025A00072B6FEE713B030BD403802400070004004
:1025B0000248016841F470010160704788ED00E055
:1025C000F0B50268274B284D284E294F294C4FF073
:1025D000804C984209D0604507D0A84205D0B0424F
:1025E00003D0B84201D0A04204D122F0700E4A6854
:1025F00042EA0E0298421BD0604519D0A84217D07B
:10260000B04215D0B84213D0A04211D01A4DA84202
:102610000ED01A4DA8420BD0194DA84208D0194D22
:10262000A84205D0184DA84202D0184DA84203D1A7
:1026300022F44075CA682A434D6922F080022A4379
:102640008D68C5620D688562984201D0A04201D1B3
:1026500009690163016841F00401016001214161E0
:102660000260F0BD0000014000040040000800408E
:10267000000C0040000401400040014000440140C3
:102680000048014000180040001C004000200040AD
:1026900010B5846842EA032224F47F440A432243AB
:1026A000826010BD826822F070020A4342F0070186
:1026B00081607047F0B5036A026A22F0010202628B
:1026C00042688469124E24F073050C682C4323F091
:1026D00002058B682B430D4DA84201D0B04205D1B5
:1026E00023F00807CB683B4323F00403A84201D042
:1026F000B04205D14D6922F4407215438A692A43DC
:1027000042608461496841630362F0BD000001409A
:1027100000040140F0B5026A036A23F0100303626B
:10272000436884690D6824F4E64444EA05248D680E
:1027300022F0200242EA05120F4D104EA84201D0AD
:10274000B04206D1CF6822F0800242EA071222F09E
:102750004002A84201D0B04207D14D6923F4406342
:1027600043EA85038D6943EA8503436084614968D0
:1027700081630262F0BD00000000014000040140DE
:10278000F0B5026A036A23F4807303624368C46984
:1027900022F4007224F073050C68124E2C438D68ED
:1027A00042EA05220E4DA84201D0B04206D1CF68C0
:1027B00022F4006242EA072222F48062A84201D099
:1027C000B04207D14D6923F4405343EA05138D69A4
:1027D00043EA05134360C4614968C1630262F0BD06
:1027E000000001400004014030B5046A026A22F48E
:1027F000805202624268C3690D6823F4E64343EAEB
:1028000005238D6824F4005444EA0534084DA84299
:1028100002D0084DA84204D14D6922F4804242EA18
:1028200085124260C36149680164046230BD0000E2
:10283000000001400004014010B5036A046A24F05E
:1028400001040462846924F0F00444EA021423F0D1
:102850000A020A438461026210BD10B5036A046A69
:1028600024F010040462846923F0A00324F470446B
:1028700044EA023243EA01118261016210BD10B5DF
:10288000806B0021C185FFF72EFA10BD01680C3165
:1028900051E8002F22F4907241E80023002BF5D17B
:1028A0000168143151E8002F22F0010241E80023B1
:1028B000002BF5D1016B012909D101680C3151E8D8
:1028C000002F22F0100241E80023002BF5D1202137
:1028D00080F8421000210163704708B590F842105B
:1028E000222901D0022008BD82684FF480539A4209
:1028F00001D1016921B1816A9A421BD04AB10AE033
:102900000268816A5268C2F308020A80816A891CDF
:1029100008E0026972B10268526802F07F020A7030
:10292000816A491C8162C18D491E0904090CC18557
:1029300003D01BE002685268F1E70168CA6822F020
:102940002002CA600168CA6822F48072CA60016805
:102950004A6922F001024A61202180F842100021D8
:102960004163026B012A03D0FFF78AFB002008BDF8
:10297000016301680C3151E8002F22F0100241E898
:102980000023002BF5D101680A68D20602D50A6837
:1029900049680091818DFFF7A5F9E7E770B5044616
:1029A00000680169E26821F4405111430161216925
:1029B000A068E26908436169114308432168CA6855
:1029C00049F20C639A430243CA6020684169A269D4
:1029D00021F440711143416131492068884202D09D
:1029E0003049884202D1FEF791FD01E0FEF77EFDFD
:1029F000E2690023192164253226B2F5004F62688E
:102A000028D0A0FB0101930F9200FDF72DFC014699
:102A1000B0FBF5F06FF01802504301EB800006EBBD
:102A20000010B0FBF5F000F0F002B1FBF5F002EBA6
:102A30000012B1FBF5F06FF01803584301EB800072
:102A400006EB0010B0FBF5F000F00F002168104419
:102A5000886070BDA0FB010192185B41FDF704FC8A
:102A60000146B0FBF5F00201B1FBF5F06FF0180381
:102A7000584301EB800006EBC000B0FBF5F000F01E
:102A8000F80002EB4002B1FBF5F0584301EB800087
:102A900006EBC000B0FBF5F000F00700D6E7000041
:102AA000001001400014014010B5044800F00AF97C
:102AB000BDE810400148FFF717B90000B40100203D
:102AC00004280AD2054A00EB400002EB00100A6815
:102AD00002604A68426009890181704758000020FD
:102AE000FEE70907090E002804DB00F1E02080F86A
:102AF0000014704700F00F0000F1E02080F8141D72
:102B00007047000000B58BB000200121CDE906011F
:102B1000089107210090CDE90201019005900490F1
:102B200069460D48FDF7AAFD0B48FEF7A9F80221FA
:102B30000948FDF733FD0E200990059069460648C7
:102B4000FDF79CFD0448FEF79BF802210248FDF7C3
:102B500025FD0BB000BD00004401002038B50F4832
:102B600000210068026842680092C26842F01002C8
:102B7000C2600A4C0A4A94F8420020280DD1322340
:102B8000A262A38561642168E06B091DFEF740FA2B
:102B90002068416941F04001416138BDB401002025
:102BA00018010020FEF776FBFFF7B8FCFFF7A4FA48
:102BB000FFF78CFAFFF768FAFFF77AFBFFF714FBD1
:102BC000FFF7CCFF1648FEF75BF8FFF7B1FBFFF706
:102BD00099FF0025FEF750FB0446401B0A281BD333
:102BE00000EE100ADFED0F0AB8EE400A20EE200AD0
:102BF000BCEEC04AFFF748FCB8EE440AFFF7C4FB3E
:102C00000948B0F90630B0F90420B0F90210B0F963
:102C10000000FDF70BFC25460120FEF71DFAD9E761
:102C2000440100206F12833A0200002070B50A8828
:102C3000C2F30A05A5F5806505804A788B78D2082D
:102C400042EA4312C2F30A04A4F5806444808A78FD
:102C5000CB78920942EA83020B7905F5257542EAA1
:102C60008322C2F30A03A3F5806383800A794E7935
:102C7000520842EAC612C2F30A02A2F58062C2807A
:102C80000E8AC6F30A06A6F5806606814E79B60955
:102C900086724979C1F30111C1724FF4A5618D4269
:102CA0000BD804F525748C4207D803F525738B42A5
:102CB00003D802F525728A4203D9002101604160E0
:102CC000816070BD18B501680A68D20624D5CA684B
:102CD000D20621D504460868486800900F4884420F
:102CE0001AD1E06B0068016821F001010160E06B1E
:102CF0000068406880B2202804D10949A1F1F4009D
:102D0000FFF794FFE16B322009684860E06B0068D0
:102D1000016841F00101016018BD0000B40100200C
:102D2000180100204FF04070E1EE100A70470006D5
:102D3000101600061016000000000000000001023E
:102D40000304060708090000000001020304000054
:102D5000702D00080000002024000000C4010008BD
:102D6000942D0008240000209C080000E0010008C9
:102D70000000000000000000000000000000000053
:102D80000000000001000000100000000000000032
:042D90000024F40027
:040000050800018965
:00000001FF
